:100000000C940D0E0C943A0E0C943A0E0C943A0E7D
:100010000C943A0E0C943A0E0C943A0E0C943A0E40
:100020000C943A0E0C943A0E0C943A0E0C943A0E30
:100030000C943A0E0C94F5CA0C943A0E0C943A0EA9
:100040000C943A0E0C9456760C943A0E0C943A0E8C
:100050000C943A0E0C943A0E0C94417F0C9440C7C9
:100060000C943A0E0C947E260C943A0E0C943A0E94
:100070000C943A0E0C943A0E0C943A0E0C943A0EE0
:100080000C943A0E0C943A0E0C943A0E0C943A0ED0
:100090000C943A0E0C943A0E0C943A0E0C943A0EC0
:1000A0000C943A0E0C943A0E0C943A0E0C943A0EB0
:1000B0000C943A0E0C943A0E0C943A0E0C943A0EA0
:1000C0000C943A0E0C943A0E0C943A0E0C943A0E90
:1000D0000C943A0E0C943A0E0C943A0E0C943A0E80
:1000E0000C943A0E084AD73B3BCE016E84BCBFFD50
:1000F000C12F3D6C74319ABD56833DDA3D00C77FF8
:1001000011BED9E4BB4C3E916BAAAABE0000008090
:100110003F05A84CCDB2D44EB93836A9020C50B91F
:10012000918688083CA6AAAA2ABE000000803F4DFE
:10013000383420582059205A20450043616E6E6F94
:100140007420656E746572207375626469723A20FA
:10015000004D3234004D3233202573006175746FC9
:1001600025692E67006572726F72207772697469F3
:100170006E6720746F2066696C65004E6F74205343
:1001800044207072696E74696E67002F00534420BA
:100190007072696E74696E67206279746520002ED2
:1001A0000044656C6574696F6E206661696C656496
:1001B0002C2046696C653A200046696C65206465B0
:1001C0006C657465643A002E006F70656E20666120
:1001D000696C65642C2046696C653A200057726929
:1001E00074696E6720746F2066696C653A20002E12
:1001F000006F70656E206661696C65642C204669CD
:100200006C653A20002E006F70656E206661696C27
:1002100065642C2046696C653A200046696C65204F
:1002200073656C6563746564002053697A653A2070
:100230000046696C65206F70656E65643A20002E1B
:10024000006F70656E206661696C65642C2046697C
:100250006C653A20004E6F77206672657368206681
:10026000696C653A20004E6F7720646F696E672075
:1002700066696C653A20002220706F73002220703E
:100280006172656E743A2200535542524F5554497B
:100290004E452043414C4C207461726765743A228C
:1002A00000747279696E6720746F2063616C6C20D2
:1002B0007375622D67636F64652066696C65732072
:1002C0007769746820746F6F206D616E79206C653A
:1002D00076656C732E204D4158206C6576656C20D8
:1002E00069733A0053442063617264206F6B006F3E
:1002F00070656E526F6F74206661696C656400761C
:100300006F6C756D652E696E6974206661696C65C8
:100310006400534420696E6974206661696C00480A
:10032000617264636F6465642044656661756C74B2
:100330002053657474696E6773204C6F61646564E3
:10034000002044002049002020204D33303120502F
:10035000005049442073657474696E67733A0020D5
:100360005A0020590020204D323036205800486F66
:100370006D65206F666673657420286D6D293A007F
:10038000204500205A002058002042002054002020
:10039000204D323035205300416476616E636564D0
:1003A000207661726961626C65733A20533D4D69D4
:1003B0006E20666565647261746520286D6D2F73AB
:1003C000292C20543D4D696E2074726176656C2035
:1003D000666565647261746520286D6D2F73292CC4
:1003E00020423D6D696E696D756D207365676D6541
:1003F0006E742074696D6520286D73292C20583D1A
:100400006D6178696D756D205859206A65726B2031
:10041000286D6D2F73292C20205A3D6D6178696DF0
:10042000756D205A206A65726B20286D6D2F7329B7
:100430002C2020453D6D6178696D756D2045206AE1
:1004400065726B20286D6D2F7329002054002020C9
:100450004D323034205300416363656C65726174C2
:10046000696F6E3A20533D616363656C65726174B8
:10047000696F6E2C20543D726574726163742061E3
:100480006363656C65726174696F6E00204500205E
:100490005A0020590020204D3230312058004D6143
:1004A00078696D756D20416363656C65726174690F
:1004B0006F6E20286D6D2F7332293A002045002081
:1004C0005A0020590020204D3230332058004D6111
:1004D00078696D756D2066656564726174657320F9
:1004E000286D6D2F73293A00204500205A002059AD
:1004F0000020204D393220580053746570732070ED
:10050000657220756E69743A004572726F723A00B6
:100510006563686F3A0053544F505045442E200095
:100520005072696E7465722073746F7070656420A8
:1005300064756520746F206572726F72732E204629
:10054000697820746865206572726F7220616E64CC
:1005500020757365204D39393920746F20726573A9
:10056000746172742E202854656D706572617475A3
:1005700072652069732072657365742E20536574EB
:10058000206974206166746572207265737461728B
:1005900074696E6729004B494C4C45442E2000502D
:1005A00072696E7465722068616C7465642E206B6C
:1005B000696C6C28292063616C6C656421006F6B29
:1005C00000526573656E643A20002200556E6B6EB2
:1005D0006F776E20636F6D6D616E643A2022005AF2
:1005E000204F6666736574203A20007A5F6D6178EB
:1005F0003A20007A5F6D696E3A20005A204F666695
:10060000736574005A204F6666736574206F6B00C3
:10061000486F74656E64206F6666736574733A0024
:100620007A5F6D61783A20007A5F6D696E3A2000DA
:10063000795F6D61783A2000795F6D696E3A2000CC
:10064000785F6D61783A2000785F6D696E3A2000BE
:10065000205A3A0020593A0020436F756E74205892
:100660003A200020453A00205A3A0020593A0058D2
:100670003A004649524D574152455F4E414D453A29
:100680004D61726C696E2056313B20537072696EF9
:100690007465722F6772626C206D6173687570206B
:1006A000666F722067656E36204649524D5741523B
:1006B000455F55524C3A68747470733A2F2F6769CE
:1006C000746875622E636F6D2F4572696B5A616C29
:1006D0006D2F4D61726C696E2F2050524F544F43F5
:1006E0004F4C5F56455253494F4E3A312E30204DB4
:1006F000414348494E455F545950453A5072696EDE
:100700007465722045585452554445525F434F55C5
:100710004E543A3320555549443A30303030303019
:1007200030302D303030302D303030302D303030D2
:10073000302D3030303030303030303030300A0012
:100740005072696E746572204F66662E0042656451
:1007500020646F6E652E0020423A0020453A005416
:100760003A004265642048656174696E672E0048EE
:10077000656174696E6720646F6E652E0020573A5C
:100780000020453A00543A0048656174696E672E4E
:100790002E2E002042403A0020403A00202F003AFE
:1007A00000205400202F0020423A00202F006F6BC1
:1007B00020543A002569206D696E2C20256920732C
:1007C000656300456E642066696C65206C697374AE
:1007D00000426567696E2066696C65206C69737498
:1007E000004E6F206D6F76652E005072696E7465D5
:1007F000722072656164792E00526573756D696E41
:1008000067207072696E74005761697420666F7238
:1008100020757365722E2E2E00536C6565702E2E1A
:100820002E00FFFFFF0000574300004D430000482B
:10083000430000A0400000A0400000004000000075
:1008400000000000000000000000000000000000A8
:1008500000000000000000574300004D4300004826
:1008600043256920686F757273202569206D696E54
:100870007574657300446F6E65207072696E74697B
:100880006E672066696C650053544F505045442E86
:1008900020005072696E7465722073746F70706599
:1008A000642064756520746F206572726F72732E98
:1008B0002046697820746865206572726F722061C5
:1008C0006E6420757365204D39393920746F20723C
:1008D0006573746172742E202854656D7065726141
:1008E000747572652069732072657365742E205368
:1008F0006574206974206166746572207265737412
:10090000617274696E6729004E6F204C696E6520B4
:100910004E756D62657220776974682063686563DF
:100920006B73756D2C204C617374204C696E653A45
:1009300020004E6F20436865636B73756D20776987
:100940007468206C696E65206E756D6265722C200E
:100950004C617374204C696E653A2000636865636E
:100960006B73756D206D69736D617463682C204CB9
:10097000617374204C696E653A20004C696E652085
:100980004E756D626572206973206E6F74204C61C4
:100990007374204C696E65204E756D6265722B31E3
:1009A0002C204C617374204C696E653A20004D31E7
:1009B000313000446F6E6520736176696E67206622
:1009C000696C652E006F6B004D3239002020506C31
:1009D000616E6E65724275666665724279746573A2
:1009E0003A20002046726565204D656D6F72793A38
:1009F00020004E6F76203132203230313500436F87
:100A00006D70696C65643A20005265705261702E99
:100A10006D6500207C20417574686F723A20004E2D
:100A20006F7620313220323031352031353A32374D
:100A30003A303900204C61737420557064617465DC
:100A4000643A2000312E302E30004D61726C696E98
:100A50000020536F66747761726520526573657408
:100A600000205761746368646F6720526573657412
:100A7000002042726F776E206F7574205265736527
:100A800074002045787465726E616C2052657365E0
:100A90007400506F776572557000737461727400E2
:100AA0002200656E717565696E67202200220065FF
:100AB0006E717565696E6720220020746F6F206CFF
:100AC0006F6E6720657874727573696F6E207072CF
:100AD0006576656E7465640020636F6C642065786C
:100AE00074727573696F6E2070726576656E746569
:100AF00064007C3C3E5E2B3D3F2F5B5D3B2C2A22FD
:100B00005C0045303A20005A3A2000593A200058FB
:100B10003A20004D53312C4D53322050696E730AE8
:100B20000024F404D9201BC40C5C0E9804C4095F93
:100B30000265077101F405F900FB04B3004804875E
:100B400000C10369005803550003034500BE023A83
:100B5000008402310053022A0029022500040220E9
:100B600000E4011C00C8011900AF0117009801142E
:100B70000084011300710110006101100051010E89
:100B80000043010D0036010B002B010B0020010B6F
:100B900000150109000C01090003010800FB000811
:100BA00000F3000800EB000700E4000600DE00068A
:100BB00000D8000600D2000600CC000500C70005E2
:100BC00000C2000500BD000400B9000400B5000427
:100BD00000B1000400AD000400A9000400A500035A
:100BE00000A20003009F0004009B00030098000384
:100BF000009500020093000300900003008D0002A6
:100C0000008B0003008800020086000200840003BD
:100C100000810002007F0002007D0002007B0002D4
:100C200000790002007700010076000200740002E3
:100C30000072000100710002006F0002006D0001EF
:100C4000006C0002006A00010069000200670001F8
:100C500000660001006500010064000200620001FE
:100C60000061000100600001005F0002005D000102
:100C7000005C0001005B0001005A00010059000106
:100C80000058000100570001005600010055000106
:100C90000054000100530000005300010052000105
:100CA0000051000100500001004F0001004E000003
:100CB000004E0001004D0001004C0001004B0000FF
:100CC000004B0001004A00010049000100480000FB
:100CD00000480001004700010046000000460001F6
:100CE00000450000004500010044000100430000F1
:100CF00000430001004200000042000100410000EA
:100D00000041000100400001003F0000003F0001E1
:100D1000003E0000003E0001003D0000003D0001DB
:100D2000003C0000003C0000003C0001003B0000D3
:100D3000003B0001003A0000003A000100390000C9
:100D400000390001003800000038000000380001C0
:100D500000370000003700010036000000360000B8
:100D600000360001003500000035000000350001AC
:100D700000340000003400000034000100330000A3
:100D80000033000000330001003200000032000098
:100D9000003200010031000000310000003100018C
:100DA000003000000030000000300001002F000083
:100DB000002F0000002F0000002F0001002E000077
:100DC000002E0000002E0001002D0000002D00006C
:100DD000002D0000002D0001002C0000002C000060
:100DE000002C0000002C0001002B0000002B000054
:100DF000002B0000002B0001002A0000002A000048
:100E0000002A0000002A000100290000002900003B
:100E1000002900000029000000290001002800002E
:100E20000028000000280000002800000028000121
:100E30000027000000270000002700000027000016
:100E40000027000100260000002600000026000008
:100E500000260000002600010025000000250000FB
:100E600000250000002500000025000000250001ED
:100E700000240000002400000024000000240000E2
:100E800000240001002300000023000000230000D4
:100E900000230000002300000023000000230001C5
:100EA00000220000002200000022000000220000BA
:100EB00000220000002200010021000000210000AB
:100EC000002100000021000000210000002100009E
:100ED0000021000100200000002000000020000090
:100EE0000020000000200000002000000020000082
:100EF00000200001001F0000001F0000001F000074
:100F0000001F0000001F0000001F0000001F000164
:100F1000001E0000001E0000001E0000001E000059
:100F20000024F4D43050C38E20C2A24017828B70AC
:100F300011127A910D816CD90AA861E108C758662F
:100F400007615143061E4B5D05C145A7041A4111B7
:100F500004093D9803713931034036DB0265339152
:100F600002D4305402802E1D02632CEE01752AC576
:100F700001B028A001102781018F2564012B244B8B
:100F800001E0223401AC211F018D200D01801FFCE6
:100F900000841EED00971DDF00B81CD200E61BC6C2
:100FA00000201BBC00641AB200B219A8000A19A0E4
:100FB000006A189900D117910040178B00B516846C
:100FC0000031167E00B31579003A157300C7146F0F
:100FD0000058146A00EE1366008813630025135E40
:100FE00000C7125B006C12570015125400C111515A
:100FF0000070114F0021114B00D61049008D104791
:10100000004610440002104200C00F4000800F3E16
:1010100000420F3C00060F3B00CB0E3800930E370A
:10102000005C0E3500270E3400F30D3200C10D3187
:1010300000900D3000600D2E00320D2D00050D2C9E
:1010400000D90C2B00AE0C2900850C29005C0C2764
:1010500000350C27000E0C2600E80B2400C40B24DE
:1010600000A00B23007D0B23005A0B2100390B211C
:1010700000180B2000F80A1F00D90A1E00BB0A1E28
:10108000009D0A1D00800A1D00630A1C00470A1B00
:10109000002C0A1B00110A1A00F7091A00DD0919B1
:1010A00000C4091900AB091900920917007B09183F
:1010B00000630917004C09160036091600200916AE
:1010C000000A091500F5081500E0081400CC081402
:1010D00000B8081400A4081400900813007D08123A
:1010E000006B08130058081200460812003408115B
:1010F00000230811001208110001081100F0071068
:1011000000E0071000D0071000C0071000B0070F64
:1011100000A107100091070E0083070F0074070F4E
:101120000065070E0057070E0049070E003B070D2C
:10113000002E070E0020070D0013070D0006070DF7
:1011400000F9060C00ED060D00E0060C00D4060CBC
:1011500000C8060C00BC060C00B0060C00A4060B70
:101160000099060C008D060B0082060B0077060B1B
:10117000006C060B0061060A0057060B004C060ABD
:101180000042060A0038060A002E060A0024060A53
:10119000001A060A001006090007060A00FD0509E4
:1011A00000F4050900EB050900E2050900D905096D
:1011B00000D0050900C7050900BE050900B50508EE
:1011C00000AD050800A50509009C05080094050868
:1011D000008C050800840508007C050800740508DB
:1011E000006C050700650508005D05070056050849
:1011F000004E0507004705070040050800380507B1
:1012000000310507002A050700230507001C050615
:1012100000160507000F0507000805060002050770
:1012200000FB040600F5040700EE040600E80406CF
:1012300000E2040700DB040600D5040600CF040624
:1012400000C9040600C3040600BD040600B7040676
:1012500000B1040500AC040600A6040600A00405C5
:10126000009B04060095040500900406008A04050E
:101270000085040500800406007A04050075040555
:1012800000700405006B0405006604050061040598
:10129000005C04050057040500520405004D0405D8
:1012A0000048040500430405003E0404003A040518
:1012B0000035040500300404002C04050027040454
:1012C00000230405001E0404001A0404001604058B
:1012D00000110404000D04040009040500040404C2
:1012E0000000040400FC030400F8030400F40304F9
:1012F00000F0030400EC030400E8030400E403042A
:1013000000E0030400DC030400D8030400D4030459
:1013100000D0030400CC030400C8030300C503038A
:1013200000656E6473746F7073206869743A205A34
:1013300000205A3A00656E6473746F707320686998
:10134000743A20590020593A00656E6473746F70C6
:1013500073206869743A20580020583A00656E641A
:1013600073746F7073206869743A20004572723A22
:10137000204D415854454D50204245440054656D20
:10138000706572617475726520686561746564204A
:10139000626564207377697463686564206F66664C
:1013A0002E204D415854454D502074726967676531
:1013B000726564202121004572723A204D494E54D5
:1013C000454D50003A2045787472756465722073FB
:1013D00077697463686564206F66662E204D494E98
:1013E00054454D50207472696767657265642021A9
:1013F000004572723A204D415854454D50003A20F4
:101400004578747275646572207377697463686572
:1014100064206F66662E204D415854454D5020740F
:101420007269676765726564202100202D20496E0E
:1014300076616C6964206578747275646572206E7B
:10144000756D626572202100504944204175746FAA
:1014500074756E652066696E6973686564212050D5
:10146000757420746865206C617374204B702C2037
:101470004B6920616E64204B6420636F6E737461EE
:101480006E74732066726F6D2061626F766520697D
:101490006E746F20436F6E66696775726174696FF1
:1014A0006E2E6800504944204175746F74756E65E6
:1014B000206661696C6564212074696D656F75745F
:1014C0000020403A006F6B20543A006F6B20423A84
:1014D00000504944204175746F74756E65206661D3
:1014E000696C6564212054656D70657261747572F4
:1014F0006520746F6F206869676800204B643A202C
:1015000000204B693A2000204B703A200020436CA9
:1015100061737369632050494420002054753A2058
:1015200000204B753A2000206D61783A2000206D34
:10153000696E3A200020643A200020626961733AA3
:10154000200070012C0190012701B0012201C0018F
:101550001D01F00118011002130130020E0160029A
:10156000090190020401C002FF000003FA004003D9
:10157000F5008003F000D003EB002004E6007004C7
:10158000E100E004DC004005D700C005D2004006C1
:10159000CD00D006C8008007C3003008BE00F008A8
:1015A000B900C009B400B00AAF00B00BAA00D00C5B
:1015B000A500000EA000500F9B00C0109600501216
:1015C000910000148C00C0158700B0178200B0197C
:1015D0007D00D01B7800001E730040206E0090221A
:1015E0006900F024640040275F0090295A00E02B36
:1015F0005500102E500020304B0010324600E033D2
:10160000410090353C001037370070383200A03967
:101610002D00B03A2800A03B2300603C1E00103D86
:101620001900903D1400103E0F00703E0A00C03EAD
:101630000500003F00002D2D3A2D2D002D2D2D00F1
:101640005344002059000120004E6F205344206372
:10165000617264005072696E742066726F6D2053FF
:10166000440053746F70207072696E740052657319
:10167000756D65207072696E7400506175736520B8
:101680007072696E7400436F6E74726F6C0050728A
:1016900065706172650054756E6500496E666F20F5
:1016A00073637265656E00052E2E004D61696E00D4
:1016B0004D3234004D3233202573004D38342058DC
:1016C0002059205A204500526573746F7265206658
:1016D00061696C73616665004D6F74696F6E00546B
:1016E000656D7065726174757265004D61696E003B
:1016F0004573746570732F6D6D00457374657073F9
:101700002F6D6D005A73746570732F6D6D005A7371
:10171000746570732F6D6D005973746570732F6DE0
:101720006D005973746570732F6D6D005873746517
:1017300070732F6D6D005873746570732F6D6D002D
:10174000412D7265747261637400412D726574720B
:1017500061637400416D6178206500416D6178209E
:101760006500416D6178207A00416D6178207A00D2
:10177000416D6178207900416D6178207900416D7B
:101780006178207800416D6178207800565472614C
:1017900076206D696E005654726176206D696E0018
:1017A000566D696E00566D696E00566D61782065E4
:1017B00000566D6178206500566D6178207A00567C
:1017C0006D6178207A00566D6178207900566D61E0
:1017D00078207900566D6178207800566D61782008
:1017E000780056652D6A65726B0056652D6A6572C4
:1017F0006B00567A2D6A65726B00567A2D6A657297
:101800006B005678792D6A65726B005678792D6A6F
:1018100065726B00416363656C00416363656C00D6
:10182000436F6E74726F6C005072656865617420EE
:1018300041425320636F6E66005072656865617443
:1018400020504C4120636F6E66005049442D430088
:101850005049442D43005049442D44005049442DE3
:1018600044005049442D49005049442D49005049F5
:10187000442D50005049442D500020022046616301
:10188000740020022046616374002002204D6178BC
:10189000002002204D6178002002204D696E00205A
:1018A00002204D696E004F6666004F6E20004F6645
:1018B00066004F6E20004175746F74656D70004650
:1018C000616E2073706565640046616E207370659B
:1018D0006564004E6F7A7A6C65004E6F7A7A6C653B
:1018E00000436F6E74726F6C004E6F7A7A6C650095
:1018F0004E6F7A7A6C650046616E20737065656420
:101900000046616E2073706565640054656D706596
:10191000726174757265004E6F7A7A6C65004E6FF5
:101920007A7A6C650046616E207370656564004666
:10193000616E2073706565640054656D70657261D9
:1019400074757265004D6F76652061786973004328
:101950006F6F6C646F776E0050726568656174209C
:10196000414253005072656865617420504C4100DB
:1019700053657420686F6D65206F66667365747358
:1019800000473238004175746F20686F6D65004DF7
:1019900038340044697361626C65207374657070DB
:1019A000657273004D61696E004D6F766520302E53
:1019B000316D6D004D6F766520316D6D004D6F7628
:1019C000652031306D6D0050726570617265004543
:1019D00078747275646572004D6F7665205A004D9B
:1019E0006F76652059004D6F76652058004D6F76F3
:1019F000652061786973004578747275646572005A
:101A00005A0059005800507265686561742041425F
:101A100053203100507265706172650050726568C4
:101A200065617420504C41203100507265706172C4
:101A30006500466C6F77203000466C6F7720300071
:101A4000466C6F7700466C6F770046616E2073704E
:101A50006565640046616E207370656564004E6F55
:101A60007A7A6C65004E6F7A7A6C650053706565A2
:101A700064005370656564004D61696E0043617276
:101A8000642072656D6F76656400436172642069DD
:101A90006E736572746564004D333030205336398F
:101AA000382050323030004D333030205336353905
:101AB00020503230300000002100240027002A008E
:101AC0002D003000330001010000040107010A016C
:101AD00000002200250028002B002E0031003400D9
:101AE00002010000050108010B0100002000230095
:101AF000260029002C002F00320000010000030105
:101B00000601090105050505070508080808020280
:101B100002020A0A08080404040401010101010187
:101B200001010303030303030303040707070C0C6A
:101B30000C0C0C0C0C0C0202020206060606060631
:101B400006060B0B0B0B0B0B0B0B010210202008D6
:101B50000810204010204080020102010804020108
:101B60000102040810204080804020100804020177
:101B700080040201804020100804020108040201D0
:101B80000102040810204080010204081020408057
:101B90000000090A02080B0C0D07060304010000EF
:101BA0000000000000000000000000000000000035
:101BB00000000000000000000000000011100F00F5
:101BC0000000000000000000000000000000000015
:101BD00000000000000002494E46494E4954594E4B
:101BE000414ECDCCCC3D0AD7233C17B7D13877CC6A
:101BF0002B329595E6241FB14F0A000020410000CA
:101C0000C84200401C4620BCBE4CCA1B0E5AAEC582
:101C10009D741227C729B3BBC22911241FBECFEF61
:101C2000D1E2DEBFCDBF00E00CBF14E0A0E0B2E027
:101C3000EAE5F7EA01E00BBF02C007900D92AE3D66
:101C4000B107D9F71BBE13E1AEEDB4E001C01D92A0
:101C5000A531B107E1F71CE1C8E1DCE104C022973E
:101C6000FE010E9453D3C231D107C9F70E944ECA68
:101C70000C94A1D30C940000A0E0B0E0E2E4FEE0FC
:101C80000C9470D3EC015B016115710519F0FB0137
:101C900091838083F9908F2D90E00E9457D3892BF8
:101CA000C9F7FDE2FF1621F4F990EE24E39405C094
:101CB0002BE2F21609F4F990EE248E010150104047
:101CC000C80167ED7BE143E050E072D2892BF9F463
:101CD0008E010E5F1F4FC8016AED7BE145E050E0C9
:101CE00067D2892B19F48E01095F1F4FA114B1042B
:101CF00019F0F50111830083E0FC04C070E090E06E
:101D000080E813C070E090E080E86FEF07C1C80181
:101D10006FED7BE143E050E04BD2892B69F4A114D5
:101D2000B10429F470E090E080EC6FE7F7C02296F0
:101D3000F501D183C083F6CF8824992440E050E098
:101D400060E070E0EF2DE053EA30A0F5F2E0EF2A1A
:101D50008E2D90E09C0128703070E2FE06C0232B8F
:101D600079F50894811C911C2BC0232B19F0089441
:101D700081089108DB01CA0112E0880F991FAA1F90
:101D8000BB1F1A95D1F7480F591F6A1F7B1F440FBD
:101D9000551F661F771F4E0F511D611D711D48395C
:101DA00029E9520729E9620729E1720748F084E02E
:101DB000E82A06C0EE3F31F4E3FC39C098E0E92A96
:101DC000F990C0CFE53311F0E53189F529912D3235
:101DD00019F4E0E1EE2A05C02B3219F081E090E021
:101DE00003C0299182E090E0E22FE053EA3018F03E
:101DF000C81BD90B1CC020E030E0FCE020383F07B6
:101E00005CF4C901880F991F880F991F280F391F8B
:101E1000220F331F2E0F311DE991E053EA3068F392
:101E2000E4FE03C0309521953F4F820E931ECE2CC9
:101E3000DD24E1FE07C0A114B10421F02197F501D2
:101E4000D183C083CB01BA010E94BCCF7B018C013E
:101E5000F3E0CF22DD2423E0C216D10421F417FBE6
:101E6000109517F9109557016801C801B70120E0D6
:101E700030E040E050E00E941CCF882309F44AC0C3
:101E800097FE0DC026EFE22E2BE1F22E9094819466
:101E900091089394C0E2D0E000E010E012C09EE010
:101EA000E92E9CE1F92EF6CFF70125913591459168
:101EB0005491C601B5010E94FCD15B016C018C1AE2
:101EC0009D0A8C169D0684F7D595C7950F5F1F4F09
:101ED0000630110529F08CEF9FEFE80EF91EF1CFC7
:101EE000C501D6017C018D018C2D880F8D2D881F99
:101EF0008F3F51F0C601B50120E030E040E050E0F6
:101F00000E941CCF882331F482E290E09093141356
:101F1000809313137E2D9F2D802F612F272F392F14
:101F2000482F562FB901CA01CDB7DEB7ECE00C94AB
:101F30008CD32F923F925F926F927F928F929F925B
:101F4000AF92BF92CF92DF92EF92FF920F931F93C7
:101F5000CF93DF938C011B01EA016115710519F024
:101F6000FB0191838083209749F0CE0102978397EC
:101F700028F020E030E040E050E0F6C0F801A19009
:101F80008F018A2D90E00E9457D3892BB9F7FDE28B
:101F9000AF1631F4F801A1908F015524539407C076
:101FA000FBE2AF1619F4F801A1908F015524209798
:101FB00019F0C031D105C1F4F0E3AF1679F4F8019E
:101FC0008081883711F0883549F4F801A1800E5FCF
:101FD0001F4FF2E05F2AC0E1D0E006C0209721F455
:101FE00080E3A816E9F427C0C830D10531F1C93023
:101FF000D10524F4C230D10531F50CC0CA30D10569
:1020000089F0C031D105F9F4C12CD12CE12CB8E014
:10201000FB2E28C0C12CD12CE12CA0E4FA2E22C02A
:10202000CAE0D0E0FCECCF2EFCECDF2EFCECEF2E77
:10203000FCE0FF2E17C0C8E0D0E0C12CD12CE12C71
:10204000E0E1FE2E0FC09E01442737FD4095542F3E
:1020500060E070E080E090E80E9414D3C901DA01EA
:102060006C017D0120E030E040E050E060E03E01A6
:10207000882477FC8094982C70EDB72EBA0CE9E098
:10208000EB1570F48A2D81548A3118F499ECB92E2D
:1020900006C08A2D81568A3150F589EAB82EBA0CCD
:1020A0008B2D90E08C179D0714F56F3FE1F0C21661
:1020B000D306E406F506B0F0CA01B901A401930104
:1020C0000E94CED29B01AC012B0D311D411D511D33
:1020D0002130F0E03F07F0E04F07F0E85F0710F431
:1020E00061E001C06FEFF801A1908F01C5CF21140D
:1020F000310481F0662331F001501040F101118369
:10210000008308C051FE1AC002501040F101118333
:10211000008314C067FF12C050FC05C02FEF3FEFD3
:102120004FEF5FE704C020E030E040E050E882E29B
:1021300090E0909314138093131316C050FE08C0C0
:1021400050954095309521953F4F4F4F5F4F0CC0B4
:1021500057FF0AC082E290E0909314138093131308
:102160002FEF3FEF4FEF5FE7B901CA01DF91CF914A
:102170001F910F91FF90EF90DF90CF90BF90AF90A5
:102180009F908F907F906F905F903F902F900895D9
:10219000FB01DC0105900D920020E1F70895FC01A0
:1021A00005900020E9F7809590958E0F9F1F089568
:1021B000FB01DC014150504088F08D9181341CF0CE
:1021C0008B350CF4805E659161341CF06B350CF43A
:1021D000605E861B611171F3990B0895881BFCCF1B
:1021E000FB01DC014150504048F005900D92002069
:1021F000C9F701C01D9241505040E0F70895FB011E
:1022000055915523A9F0BF01DC014D9145174111AE
:10221000E1F759F4CD010590002049F04D914015AA
:102220004111C9F3FB014111EFCF81E090E001972B
:102230000895FB01DC0104C08D910190801921F407
:1022400041505040C8F7881B990B0895FB01DC01F1
:1022500002C001900D9241505040D8F70895FB0103
:10226000DC018D9181341CF08B350CF4805E619122
:1022700061341CF06B350CF4605E861B611189F3D0
:10228000990B0895FB01DC010D900020E9F71197EF
:1022900001900D920020E1F70895FC0181918617CD
:1022A00021F08823D9F7992708953197CF01089510
:1022B000FB01DC018D91019080190110D9F3990B7C
:1022C0000895FB01DC0101900D920020E1F70895D3
:1022D000FB01DC014150504030F08D91019080199C
:1022E00019F40020B9F7881B990B0895FB01DC0154
:1022F0004150504048F001900D920020C9F701C0B4
:102300001D9241505040E0F70895AEE0B0E0EBE898
:10231000F1E10C9478D30E891F898EE08C831A83A7
:1023200009838FEF9FE79E838D839E01265E3F4F3B
:10233000CE010196688D798DA9010AD02F8138854B
:10234000020F131FF80110822E96E4E00C9494D330
:10235000ABE0B0E0EEEAF1E10C946AD33C012B0172
:102360005A01FC0117821682838181FD03C06FEF41
:102370007FEFB9C19AE0892E1E010894211C311CFF
:10238000F3012381F20123FD859123FF81912F0128
:10239000882309F4A5C1853239F423FD859123FFF3
:1023A00081912F01853221F490E0B301B7D1E8CFBC
:1023B000982FFF24EE249924FFE1FF15D0F09B32E3
:1023C00069F09C3228F4903259F0933291F40EC0A7
:1023D0009D3249F0903369F441E024C052E0F52A7F
:1023E00084E0F82A28C098E0F92A25C0E0E1FE2A16
:1023F00022C0F7FC29C0892F80538A3070F4F6FE82
:1024000005C0989C902C1124980E15C0E89CE02CD7
:102410001124E80EF0E2FF2A0EC09E3229F4F6FCE9
:102420005FC140E4F42A07C09C3619F450E8F52A4D
:1024300002C0983649F4F20123FD959123FF919152
:102440002F01992309F0B8CF892F8554833018F0D4
:102450008052833038F444E050E0A40EB51E5FE3B0
:1024600059830FC0933631F0933779F0933509F0E3
:1024700052C01FC0F5018081898342E050E0A40E64
:10248000B51E610101E010E011C0F501C080D180EE
:10249000F6FC03C06FEF7FEF02C0692D70E042E0F1
:1024A00050E0A40EB51EC6012ED18C015FE7F522C7
:1024B00013C0F501C080D180F6FC03C06FEF7FEF41
:1024C00002C0692D70E042E050E0A40EB51EC601C6
:1024D0000FD18C0150E8F52AF3FE06C018C080E247
:1024E00090E0B3011BD1EA948E2D90E008171907F4
:1024F000B0F30DC0F601F7FC8591F7FE81916F01F5
:1025000090E0B3010BD1E110EA94015010400115A5
:10251000110581F7E2C0943611F0993661F5F7FEA6
:1025200008C0F501208131814281538184E090E02F
:102530000AC0F501808191819C01442737FD4095B7
:10254000542F82E090E0A80EB91E9FE6F92257FFB3
:1025500009C050954095309521953F4F4F4F5F4FA3
:10256000E0E8FE2ACA01B901A1012AE030E002D167
:10257000D82ED2183FC0953729F41F2D1F7E2AE090
:1025800030E01DC01F2D197F9F3661F0903720F479
:10259000983509F0A5C00FC0903739F0983709F089
:1025A0009FC004C028E030E00AC0106114FD146030
:1025B00020E130E004C014FD166020E132E017FF96
:1025C00008C0F501608171818281938144E050E00F
:1025D00008C0F50180819181BC0180E090E042E07B
:1025E00050E0A40EB51EA101C5D0D82ED2188FE799
:1025F000F82EF122F6FE0BC05EEFF522D91438F466
:10260000F4FE07C0F2FC05C08FEEF82202C01D2DBB
:1026100001C0192DF4FE0DC0FE01ED0DF11D8081EC
:10262000803319F499EEF92208C01F5FF2FE05C04D
:1026300003C08F2D867809F01F5F0F2DF3FC13C0A8
:10264000F0FE0EC01E1510F09D2C0AC09D2C9E0C95
:10265000911A1E2D05C080E290E0B3015FD01F5F8C
:102660001E15C8F304C01E1510F4E11A01C0EE24B3
:1026700004FF0EC080E390E0B30150D002FF1BC006
:1026800001FD03C088E790E00EC088E590E00BC034
:10269000802F867881F001FF02C08BE201C080E2CA
:1026A000F7FC8DE290E0B30139D005C080E390E003
:1026B000B30134D09A94D914C8F3DA94F101ED0D32
:1026C000F11D808190E0B30129D0DD20B1F705C074
:1026D00080E290E0B30122D0EA94EE20C9F750CE18
:1026E000F30166817781CB012B96E2E10C9486D3CE
:1026F000FC010590615070400110D8F780959095CD
:102700008E0F9F1F0895FC016150704001900110D1
:10271000D8F7809590958E0F9F1F08950F931F9364
:10272000CF93DF938C01EB018B8181FF1BC082FF74
:102730000DC02E813F818C819D812817390764F45B
:10274000E881F9810193F983E88306C0E885F9857A
:10275000802F1995892B31F48E819F8101969F835B
:102760008E8302C00FEF1FEFC801DF91CF911F9141
:102770000F910895FA01AA27283051F1203181F1F3
:10278000E8946F936E7F6E5F7F4F8F4F9F4FAF4F79
:10279000B1E03ED0B4E03CD0670F781F891F9A1F8C
:1027A000A11D680F791F8A1F911DA11D6A0F711D40
:1027B000811D911DA11D20D009F468943F912AE04C
:1027C000269F11243019305D3193DEF6CF01089534
:1027D000462F4770405D4193B3E00FD0C9F7F6CF65
:1027E000462F4F70405D4A3318F0495D31FD40522D
:1027F000419302D0A9F7EACFB4E0A69597958795C3
:1028000077956795BA95C9F70097610571050895A1
:102810009B01AC010A2E069457954795379527954D
:10282000BA95C9F7620F731F841F951FA01D0895E5
:10283000FC01128213820895FC018381882311F028
:1028400081E082830895FC018281811112820895C2
:10285000CF93DF93DC01FC01EB55FE4F808191812A
:102860000097C9F1019791838083ED01CC5ADF4F26
:10287000FD01ED58FF4F8BE1019009928150E1F786
:10288000FD01EE5AFF4FAF58BF4F8D919C911197AC
:10289000A157B04091838083FD01ED58FF4F20E0A8
:1028A00030E0AD014B555E4F10C02F5F3F4FEF0141
:1028B000DF015F968BE10D9009928150E1F7858DE4
:1028C000968D329791838083B196DA018D919C9198
:1028D0002817390750F3DF91CF910895FC0188E75D
:1028E00094E0918380838781882321F0CF0104962F
:1028F0000C9424680895CF92DF92EF92FF920F9389
:102900001F93DF93CF93CDB7DEB76F970FB6F894D1
:10291000DEBF0FBECDBF8C016B01095A1F4FD8011E
:102920008C9107551040882321F42FE2E22EF12CE0
:1029300003C090E5E92EF12CE00EF11E88E794E04B
:102940009A8389831C821B8218861D82B7016C5F63
:102950007F4FCE010596A60121E00E94106F8823CB
:1029600091F5E0E1F5E0949108C08091C00085FF09
:10297000FCCF9093C600319694919923B1F7EBE385
:10298000F1E0949108C08091C00085FFFCCF909346
:10299000C600319694919923B1F709C08091C00087
:1029A00085FFFCCF0894C11CD11C9093C600F60192
:1029B0009081992399F78091C00085FFFCCF8AE030
:1029C0008093C6005AC0F801EB55FE4F208131813B
:1029D0002A30310508F040C02F5F3F4F31832083FC
:1029E00021503040F90185E0EE0FFF1F8A95E1F795
:1029F000E21BF30BED58FF4FE00FF11F13C0AF01C7
:102A0000415E5F4FBF018BE1DB010D90BD01DA013B
:102A10000D92AD018150C1F7929182913296968FBD
:102A2000858F7F9721503040BFEF2E3F3B0739F70E
:102A3000D801AD58BF4FF70134968BE101900D924C
:102A40008150E1F70F581F4FF70182819381D80120
:102A50008D939C9301571040D801AC5ABF4FFE0193
:102A600035968BE101900D928150E1F70E5A1F4F80
:102A70008B819C81F80191838083CE0101962EDFAA
:102A80006F960FB6F894DEBF0FBECDBFCF91DF912A
:102A90001F910F91FF90EF90DF90CF900895EF92EC
:102AA000FF920F931F938C013EECE32E31E0F32E47
:102AB000E80EF91EC7010E94D767C7010E9424686B
:102AC000F801108211821F910F91FF90EF900895ED
:102AD000CF92DF92EF92FF920F931F93CF93DF93EA
:102AE0007C016B01DB010D900020E9F78D010150A5
:102AF0001040061B170BEEECF1E0EE0EFF1ED701A7
:102B00001C92E2E3FEEFEE0EFF1ECB016EE470E0DE
:102B1000C4DBEC01009731F4F8013197EC0DFD1D99
:102B200086010CC060E270E0B8DB8C010F5F1F4FC4
:102B3000CE016AE270E0B1DBFC0131978DE0818368
:102B40008AE082831382C70186539E4FB8010E9498
:102B500021708EEC91E0E80EF91ED7018C9188234C
:102B600019F1E9E0F5E0949108C08091C00085FF7B
:102B7000FCCF9093C600319694919923B1F7E5E686
:102B8000F1E0949108C08091C00085FFFCCF909344
:102B9000C600319694919923B1F78091C00085FFCA
:102BA000FCCF8AE08093C600DF91CF911F910F91F7
:102BB000FF90EF90DF90CF900895CF93DF93EC01DB
:102BC0008B81882309F43BC0EDE8F1E0949108C0C3
:102BD0008091C00085FFFCCF9093C6003196949100
:102BE0009923B1F7CD57DD4F488159816A817B81A7
:102BF000C358D24082E695E02AE030E00E94AB273D
:102C0000EBE8F1E0949108C08091C00085FFFCCF13
:102C10009093C600319694919923B1F7C558DD4F32
:102C2000488159816A817B8182E695E02AE030E023
:102C30000E94AB278091C00085FFFCCF12C0EBE75C
:102C4000F1E0949108C08091C00085FFFCCF909383
:102C5000C600319694919923B1F78091C00085FF09
:102C6000FCCF8AE08093C600DF91CF9108952F9228
:102C70003F924F925F926F927F928F929F92AF920C
:102C8000BF92CF92DF92EF92FF920F931F93DF9349
:102C9000CF93CDB7DEB7AC970FB6F894DEBF0FBEBB
:102CA000CDBF5C014B01FC018381882309F43BC14A
:102CB000C50182539E4F0E942468F50112821A8A30
:102CC0001D8A198A188A88E794E09F878E875EE4B8
:102CD000C52ED12CCA0CDB1C2FE230E0A20EB31E95
:102CE000F601B182A08221ED3FEFA20EB31EF401E6
:102CF00080818F3209F08DC0C4016FE270E0CDDABF
:102D00007C010894E11CF11C3E010894611C711CBB
:102D1000260142E1242E312C2C0E3D1E75C0C70128
:102D20006FE270E0BADA6C01009709F480C0E8162F
:102D3000F90608F07CC08C010E191F09C301B70108
:102D4000A801D4DA060D171DF8011082F30107C09F
:102D50008091C00085FFFCCF31969093C600908192
:102D60009923B1F78091C00085FFFCCFFAE0F09382
:102D7000C600F201608171816115710519F460E08E
:102D800070E002C06C5F7F4FC101A30121E00E948F
:102D9000106F882371F5E9ECF1E0949108C08091FF
:102DA000C00085FFFCCF9093C60031969491992383
:102DB000B1F7FE01319607C08091C00085FFFCCFBE
:102DC00031969093C60090819923B1F7E7ECF1E03A
:102DD000949108C08091C00085FFFCCF9093C600FD
:102DE000319694919923B1F78091C00085FFFCCF73
:102DF00094C02EE030E02C0F3D1FF2013183208380
:102E000076010894E11CF11CE114F10409F087CF6C
:102E10000BC080E590E0A80EB91EF601B182A08239
:102E200020EB3FEFA20EB31ED82C092D02C0DE2CE2
:102E30000F2D8EE490E0A80EB91EF50180819181DE
:102E400022EB3FEFA20EB31E009719F480E090E052
:102E500001C004966D2D702F0E94DC6F882371F1E4
:102E6000E9EBF1E0949108C08091C00085FFFCCFB0
:102E70009093C600319694919923B1F78D2D902FA0
:102E80009C01F90107C08091C00085FFFCCF3196FD
:102E90009093C60090819923B1F78091C00085FF7F
:102EA000FCCF8AE08093C60083E892E0A80EB91EAA
:102EB000F501108211821282138232C0E1EAF1E040
:102EC000949108C08091C00085FFFCCF9093C6000C
:102ED000319694919923B1F78D2D902F9C01F90192
:102EE00007C08091C00085FFFCCF31969093C6004B
:102EF00090819923B1F7EFE9F1E0949108C08091B6
:102F0000C00085FFFCCF9093C60031969491992321
:102F1000B1F78091C00085FFFCCF8AE08093C600A6
:102F2000CE010E96DBDCAC960FB6F894DEBF0FBE7A
:102F3000CDBFCF91DF911F910F91FF90EF90DF9068
:102F4000CF90BF90AF909F908F907F906F905F9049
:102F50004F903F902F900895BF92CF92DF92EF92C3
:102F6000FF920F931F93CF93DF938C01EB018FE2BE
:102F70008993EE24E394FF2475EAC72E71E0D72EDF
:102F8000C00ED11E6FE1B62E14C0FB9CC0011124EF
:102F90008D589F4F800F911FBE010E94346802C060
:102FA0002196E3948881882319F08CE88E15C0F768
:102FB000F3942F2D30E0F601808191812817390795
:102FC00020F3E7FC07C0C80182539E4FBE010E9458
:102FD000346801C01882DF91CF911F910F91FF904B
:102FE000EF90DF90CF90BF900895EF92FF920F93F4
:102FF0001F93CF93DF938C01FC01138286A9882352
:1030000021F0C801C3960E942468E7EAEE2EE1E0B1
:10301000FE2EE00EF11EC70160E045E30E94D3657D
:10302000882309F5E0E1F5E0949108C08091C000A3
:1030300085FFFCCF9093C600319694919923B1F708
:10304000E2E1F3E0949108C08091C00085FFFCCFDD
:103050009093C600319694919923B1F78091C00066
:1030600085FFFCCF7DC0E801C455DE4FCE01B7011E
:1030700041E00E94B270882341F5CE01B70140E0E3
:103080000E94B270882309F5E9E0F5E0949108C048
:103090008091C00085FFFCCF9093C600319694913B
:1030A0009923B1F7EFEFF2E0949108C08091C0004E
:1030B00085FFFCCF9093C600319694919923B1F788
:1030C0008091C00085FFFCCF4BC0C801C396BE01F4
:1030D0000E94166B882309F5E9E0F5E0949108C099
:1030E0008091C00085FFFCCF9093C60031969491EB
:1030F0009923B1F7EFEEF2E0949108C08091C000FF
:1031000085FFFCCF9093C600319694919923B1F737
:103110008091C00085FFFCCF23C081E0F80183834C
:10312000E0E1F5E0949108C08091C00085FFFCCFFC
:103130009093C600319694919923B1F7E4EEF2E0B2
:10314000949108C08091C00085FFFCCF9093C60089
:10315000319694919923B1F78091C00085FFFCCFFF
:103160008AE08093C600D801AC5ABF4FF801F396AD
:103170008BE101900D928150E1F7F80181A992A9AC
:103180000E5A1F4FF8019183808302551040C801E9
:103190008F96025B1F4FF80191838083DF91CF915F
:1031A0001F910F91FF90EF9008952F923F924F92B1
:1031B0005F926F927F929F92AF92BF92CF92DF9277
:1031C000EF92FF920F931F93DF93CF93CDB7DEB7AC
:1031D000CC55D0400FB6F894DEBF0FBECDBF6C010A
:1031E000662311F527E832E0C20ED31ED6018C917A
:1031F000E9E7FDEFCE0EDF1E882309F4E2C02FE7DA
:1032000032E0C20ED31ED601ED90FD900D911C91BF
:10321000E1E8FDEFCE0EDF1E0E9488C7E616F70636
:103220000807190708F4CDC027E832E0C20ED31E04
:10323000D6011C92E9E7FDEFCE0EDF1ED6011396F4
:103240008C91882339F4C601D0DEF601838188236E
:1032500009F4B7C000D000D0EDB7FEB731967E01BB
:103260000894E11CF11CADB7BEB71296FC92EE9229
:1032700011978CE591E093838283D6019D968D9181
:103280009C919E979583848340D88701EDB7FEB7C4
:1032900036960FB6F894FEBF0FBEEDBF57010AC0B9
:1032A000D8018C91992787FD90950E945FD3F801F2
:1032B00081938F01F50101900020E9F73197EA1918
:1032C000FB09802F8E198E175CF313E3A12EB12C0E
:1032D000AC0CBD1CC50140E050E060E070E00E9415
:1032E0000D679924BDE3EB2EF12CEC0EFD1E2E0193
:1032F0000894411C511CAFE16A2E712C6C0E7D1E8E
:10330000F5E52F2EF1E03F2E42C0D8018C9190E0E0
:103310000E945FD3F80181938F01D7010D900020A7
:10332000E9F71197AE19BF09802F8E198A176CF330
:1033300027968FAD27978E3751F1C701B20145E02F
:1033400050E00E946811009711F500D000D0EDB751
:10335000FEB73196ADB7BEB712967C926E921197BA
:1033600033822282558244820E948511EDB7FEB7D6
:1033700036960FB6F894FEBF0FBEEDBFC3010E9494
:103380001F4B81E591E00E94A64A99249394C501C0
:10339000B70140E050E00E94356A181614F4870126
:1033A000BCCF992041F48FEF9FEFD6019E969C935E
:1033B0008E939D9706C0F60185A596A5019696A7C2
:1033C00085A7C45ADF4F0FB6F894DEBF0FBECDBF3E
:1033D000CF91DF911F910F91FF90EF90DF90CF90F1
:1033E000BF90AF909F907F906F905F904F903F9075
:1033F0002F9008952F923F924F925F926F927F92FB
:103400008F929F92AF92BF92CF92DF92EF92FF92F4
:103410000F931F93DF93CF93CDB7DEB7CF58D04034
:103420000FB6F894DEBF0FBECDBF8C012B016A0131
:10343000C757DF4F39832883C958D04084E090E0D4
:10344000C80ED91EF8017196C957DF4FF983E8837A
:10345000C758D04044E0642E712C600E711ECA57CC
:10346000DF4F1882C658D04036E6E32EF12CEC0E22
:10347000FD1EC7010B96C557DF4F99838883CB5834
:10348000D04028E8822E22E0922E800E911E9AE8EB
:10349000A92E92E0B92EA00EB11E87E4282E312C61
:1034A0002C0E3D1EF1013496C357DF4FF983E8839C
:1034B000CD58D040E0E1F5E08491C157DF4F8883DB
:1034C000CF58D04053C1F7018385482F50E0BA014F
:1034D000687170706031710509F056C1F401208186
:1034E00031812130310509F44FC12230310509F411
:1034F0004BC1F701DE0111969081903239F08E2F89
:103500008E19883011F48EE28D939D933196C557B4
:10351000DF4F88819981CB58D040E817F90761F7D0
:103520001C921E86F2018081882331F4CE010E9612
:1035300060E072E00E944211CE010E96B2010E943C
:103540004211CE010E96BE016F5F7F4F0E94421165
:10355000CE010E9660E072E00E9442111CA61FA6EA
:103560001BA61AA688E794E099A788A7CE018C9697
:10357000B601AE014F5F5F4F21E00E94106F8823BC
:1035800009F03FC0F40180819181892BD1F5C157A9
:10359000DF4F9881CF58D040E0E1F5E008C080913E
:1035A000C00085FFFCCF9093C6003196949199237B
:1035B000B1F7E2E0F2E007C08091C00085FFFCCFE8
:1035C00031969093C60090819923B1F78091C00005
:1035D00085FFFCCFFAE0F093C600FE01319607C0EC
:1035E0008091C00085FFFCCF31969093C6009081FA
:1035F0009923B1F78091C00085FFFCCF8AE08093CA
:10360000C600C357DF4FA881B981CD58D040FE0115
:10361000BC968BE101900D928150E1F78AA59BA5A4
:10362000F1019383828388E794E091838083C801CA
:10363000BE01625F7F4FA10120E030E0DBDEC1010F
:103640004DD9CE0188964AD991C09E3209F48EC0D8
:103650009F3509F48BC0F80191899E3209F486C028
:103660009F3509F483C043FD81C080E0603171055E
:1036700009F481E0F80184A7882349F4F7018085E3
:10368000873409F073C081858E3709F46FC0D30188
:10369000F7018081803241F08E2F8E19883011F42D
:1036A0008EE28D9380818D933196C557DF4F88814F
:1036B0009981CB58D040E817F90759F71C92F401CB
:1036C00080819181009701F5F20107C08091C000CF
:1036D00085FFFCCF31969093C60090819923B1F776
:1036E000F30107C08091C00085FFFCCF3196909315
:1036F000C60090819923B1F78091C00085FFFCCF6F
:10370000FAE0F093C60032C08130910539F4F5013A
:103710008081918101969183808328C0029731F541
:10372000C757DF4F88819981C958D040009731F041
:10373000B3010E942F11892B71F42BC0CA57DF4FA0
:103740009881C658D040292F30E0F50180819181C1
:1037500028173907F1F0CA57DF4FF881C658D04013
:10376000FF5FCA57DF4FF883C658D040C601B70184
:10377000C957DF4F48815981C758D0400E94356AE8
:1037800018160CF4A0CE05C0F7019081992309F01A
:103790005CCFC157DF4F0FB6F894DEBF0FBECDBF71
:1037A000CF91DF911F910F91FF90EF90DF90CF901D
:1037B000BF90AF909F908F907F906F905F904F9051
:1037C0003F902F900895EF92FF920F931F93DF93F6
:1037D000CF93CDB7DEB76F970FB6F894DEBF0FBEAD
:1037E000CDBF7C018C01025B1F4F805B9F4FF801B6
:1037F0009183808328E832E0E20EF31E21E030E07E
:10380000F701219331937F011182108226E73DEF6A
:10381000E20EF31E049640E050E060E070E00E948B
:103820000D67F80120813181DE011596F90134968A
:103830008BE101900D928150E1F7F9018281938132
:103840009C838B8388E794E09A838983C70165E131
:1038500072E08E010F5F1F4FA80120E030E0CADD4B
:10386000C8013CD8F701E657FD4F808191816F96E2
:103870000FB6F894DEBF0FBECDBFCF91DF911F9181
:103880000F91FF90EF900895CF92DF92EF92FF9209
:103890000F931F93DF93CF93CDB7DEB76F970FB61C
:1038A000F894DEBF0FBECDBF7C016A018C01025BC4
:1038B0001F4F805B9F4FF8019183808328E832E09F
:1038C000E20EF31E22E030E0F701219331937F01F5
:1038D0007183608326E73DEFE20EF31E049640E01D
:1038E00050E060E070E00E940D67F80120813181B6
:1038F000DE011596F90134968BE101900D9281500D
:10390000E1F7F901828193819C838B8388E794E0BE
:103910009A838983C70165E172E08E010F5F1F4FB3
:10392000A801960167DDC8010E946E146F960FB65C
:10393000F894DEBF0FBECDBFCF91DF911F910F91E5
:10394000FF90EF90DF90CF9008952F923F924F928B
:103950005F926F927F928F929F92AF92BF92CF921F
:10396000DF92EF92FF920F931F93DF93CF93CDB728
:10397000DEB7AD970FB6F894DEBF0FBECDBF7C01AA
:103980003B014DA7DC0113968C91882309F450C3A9
:10399000E1EDF1E0EE0EFF1ED7018C91EFE2FEEFBC
:1039A000EE0EFF1E882309F418C1222309F0E0C09F
:1039B00029EE31E0E20EF31ED7018C91E7E1FEEF34
:1039C000EE0EFF1E882371F1E9E0F5E0949108C046
:1039D0008091C00085FFFCCF9093C60031969491F2
:1039E0009923B1F7E1EAF2E0949108C08091C00018
:1039F00085FFFCCF9093C600319694919923B1F73F
:103A000082E695E061E070E04AE050E00E94FA272B
:103A10008091C00085FFFCCF8AE08093C6000E94A1
:103A20000E2A06C3E0E1F5E0949108C08091C00041
:103A300085FFFCCF9093C600319694919923B1F7FE
:103A4000E8E8F2E0949108C08091C00085FFFCCFC7
:103A50009093C600319694919923B1F7F30107C072
:103A60008091C00085FFFCCF31969093C600908175
:103A70009923B1F7EDE7F2E0949108C08091C0007E
:103A800085FFFCCF9093C600319694919923B1F7AE
:103A9000C7012EEE31E0E20EF31EB7015DDA4BEF07
:103AA0005FEFE40EF51ED7019C91E7E1FEEFEE0E0D
:103AB000FF1E8DE8989FF0011124E251FE4FEE0D9C
:103AC000FF1D07C08091C00085FFFCCF3196909309
:103AD000C60090819923B1F7E7E7F2E0949108C01E
:103AE0008091C00085FFFCCF9093C60031969491E1
:103AF0009923B1F723E832E0E20EF31ED7014D918E
:103B00005D916D917C91EDE7FDEFEE0EFF1E82E67B
:103B100095E02AE030E00E94AB278091C00085FF4D
:103B2000FCCF8AE08093C600A70147515E4FDA01BF
:103B30002C91E22FF0E0EE0FFF1FEE0FFF1FEE0DB6
:103B4000FF1DE651FE4F83E892E0E80EF91ED70113
:103B5000AD90BD90CD90DC908DE79DEFE80EF91E05
:103B6000A082B182C282D3822F5FDA012C932FC050
:103B7000E0E1F5E0949108C08091C00085FFFCCFA2
:103B80009093C600319694919923B1F7E6E6F2E05E
:103B9000949108C08091C00085FFFCCF9093C6002F
:103BA000319694919923B1F7F30107C08091C00039
:103BB00085FFFCCF31969093C60090819923B1F791
:103BC0008091C00085FFFCCF8AE08093C600C701CA
:103BD00082539E4F0E94246839C0E9EEF1E0EE0E58
:103BE000FF1ED7011C92E7E1FEEFEE0EFF1EE0E1A3
:103BF000F5E0949108C08091C00085FFFCCF9093C0
:103C0000C600319694919923B1F7E5E5F2E09491DD
:103C100008C08091C00085FFFCCF9093C60031960C
:103C200094919923B1F7F30107C08091C00085FFFB
:103C3000FCCF31969093C60090819923B1F7809183
:103C4000C00085FFFCCF8AE08093C600D7011296A2
:103C50001C921A8A1D8A198A188A88E794E09F871D
:103C60008E876EE4A62EB12CAE0CBF1CEFE2F0E006
:103C7000EE0EFF1ED501ED92FC92E1EDFFEFEE0E90
:103C8000FF1ED3018C918F3209F090C0C3016FE207
:103C900070E00E944D116C010894C11CD11C4E01B2
:103CA0000894811C911C250152E1252E312C2C0EEB
:103CB0003D1E77C0C6016FE270E00E944D115C01AD
:103CC000009709F480C0C816D90608F07CC08C01A2
:103CD0000C191D09C401B601A8010E947611080D36
:103CE000191DF8011082F40107C08091C00085FF02
:103CF000FCCF31969093C60090819923B1F78091C3
:103D0000C00085FFFCCFFAE0F093C600D2016D91B0
:103D10007C916115710519F460E070E002C06C5F80
:103D20007F4FC101A40121E00E94106F882371F52B
:103D3000E1E4F2E0949108C08091C00085FFFCCFDF
:103D40009093C600319694919923B1F7FE01319674
:103D500007C08091C00085FFFCCF31969093C600CC
:103D600090819923B1F7EFE3F2E0949108C080913C
:103D7000C00085FFFCCF9093C600319694919923A3
:103D8000B1F78091C00085FFFCCF23C12EE030E069
:103D90002C0F3D1FF2013183208365010894C11C63
:103DA000D11CC114D10409F085CF0BC040E550E00F
:103DB000E40EF51ED501ED92FC92E0EBFFEFEE0E66
:103DC000FF1E830101C08601F701E25BFF4F2DA5B5
:103DD000222309F4BFC0608171816115710519F456
:103DE00060E070E002C06C5F7F4FC70182539E4F5E
:103DF000A80121E00E94106F882309F47EC04FEDD6
:103E000051E0E40EF51ED7014D915D916D917C91CD
:103E1000ECE9F0E0EE0EFF1ED7014D935D936D933C
:103E20007C931397E5E8FDEFEE0EFF1EE1E3F2E071
:103E3000949108C08091C00085FFFCCF9093C6008C
:103E4000319694919923B1F7F80107C08091C00091
:103E500085FFFCCF31969093C60090819923B1F7EE
:103E6000E9E2F2E0949108C08091C00085FFFCCFA8
:103E70009093C600319694919923B1F782E695E02C
